:0200000480007A
:100000006F00C004732F2034930F8000630AFF0336
:10001000930F90006306FF03930FB0006302FF038A
:10002000170F0080130F0FFE63040F0067000F000F
:10003000732F203463540F006F004000136E9E53E3
:10004000171F00002320CFFD6FF09FFF732540F1A5
:100050006310050073251030635805000F00F00F82
:10006000130E100073000000130E00009702000032
:10007000938282F973905230735020307350303035
:1000800073504030970200809382C2F7638C020065
:10009000739052109302B01A739022307323203061
:1000A000E39E62F873500030970200009382420191
:1000B00073901234732540F1730020309300400197
:1000C00013016000B3D12002930E3000130E200004
:1000D0006396D10D9300C0FE13016000B3D12002DE
:1000E000B7BEAA2A938E7EAA130E30006398D10B56
:1000F000930040011301A0FFB3D12002930E000032
:10010000130E4000639CD1099300C0FE1301A0FFB1
:10011000B3D12002930E0000130E50006390D1095A
:10012000B700008013011000B3D12002B70E008089
:10013000130E60006394D107B70000801301F0FF35
:10014000B3D12002930E0000130E70006398D10506
:10015000B700008013010000B3D12002930EF0FF1E
:10016000130E8000639CD103930010001301000064
:10017000B3D12002930EF0FF130E90006390D103D1
:100180009300000013010000B3D12002930EF0FF92
:10019000130EA0006394D101631CC0010F00F00F87
:1001A00063000E00131E1E00136E1E00730000007D
:1001B0000F00F00F130E100073000000731000C04A
:0401C000000000003B
:1010000000000000000000000000000000000000E0
:1010100000000000000000000000000000000000D0
:1010200000000000000000000000000000000000C0
:1010300000000000000000000000000000000000B0
:081040000000000000000000A8
:040000058000200057
:00000001FF
